:10000000000003308A00022B8030A100FE30E22085
:100010000130E2207530AF0030301629A101A11760
:10002000BD00FE30E2203D08E228C900C01F1A28AA
:100030002D30E220A601A701A801A901C0176A304E
:10004000BF070310C00CC10CC20CA90CA80CA70C54
:10005000A60CBF0F212842083F02C207BF02410879
:100060004002C107C002A5016D202E30E220CA0166
:100070000310260DC200270DC100280DC000290D58
:10008000BF00CA0D0310C20DC10DC00DBF0DCA0DBA
:100090002608C20727080318270FC10728080318D6
:1000A000280FC00729080318290FBF070318CA0F14
:1000B0000310C20DC10DC00DBF0DCA0D4A08303E60
:1000C000E2204208A6004108A7004008A8003F0817
:1000D000A900C90B37280310BF29A0112508031D4B
:1000E0007428A0150A30A5004208B1004108B000EC
:1000F0004008AF003F08AE00A401B901B801B70144
:100100000A30B6002921A40A24082502031D7D28EF
:100110003608031DA011A01D8F28250B9228360834
:10012000303EE220A50B7428BF29BB0087110613BF
:100130008316871106130F30870583123B08A0181A
:10014000BF283E30AF00803016213330BA00D320B4
:100150001330AF0088301621D32064301521D3200E
:10016000643015212230BA00D3202830BE200C3054
:10017000BE200630BE20A0143B08BF282014BA00C1
:10018000201CCD280613033C031CD228D2200730A4
:10019000AF00D0301621031408002014FE3C0319D0
:1001A000E0280617201C201087150F3087053A0815
:1001B000F03987048711BA0E2018D3283230152160
:1001C0003B08BF29A11B95280800A400A201240810
:1001D00003178D000313250803178F00F820031958
:1001E000BF29E220A40A0319A50AA20FE728BF2904
:1001F000831603178C170C140000000083120C08E0
:10020000BF2983178001840AFF3E031D0229BF29ED
:10021000B301B200FF30B207031CB307031CBF29B0
:100220000330AF00E43016210A29AF01F43EAE00DE
:10023000AF09FE30031C1F29AE0703181C29AE07A7
:100240000000AF0F1C2900002E1826292E1828297F
:100250000800310839068039BB00B11F3A29AE09C0
:10026000AF09B009B109AE0A0319AF0A0319B00A00
:100270000319B10AB91F4729B609B709B809B9095D
:10028000B60A0319B70A0319B80A0319B90AB20161
:10029000B301B401B501C301C401C501C6013908E8
:1002A000380437043604031985292030BA000310B6
:1002B000AE0DAF0DB00DB10DC30DC40DC50DC60D06
:1002C00039084602031D6E2938084502031D6E29B0
:1002D00037084402031D6E2936084302031C7F2998
:1002E0003608C3023708031C370FC4023808031C42
:1002F000380FC5023908031C390FC6020314B20DAA
:10030000B30DB40DB50DBA0B5729BB1F9229B20915
:10031000B309B409B509B20A0319B30A0319B40A37
:100320000319B50A4308B6004408B7004508B800E9
:100330004608B9003208AE003308AF003408B000F8
:100340003508B100BF29B701B6011030BA002F0D32
:10035000B60DB70D3208B6023308031C330FB702CF
:100360000318B9293208B60733080318330FB70743
:100370000310AE0DAF0DBA0BA7292E08BF298313AA
:1003800083120313000008002B082706CD00CD1BA5
:10039000F929AB1BE2292A082602031C0034031D9D
:1003A00001342B082702031C0034031D01342C08E0
:1003B0002802031C0034031D01342D082902031CEC
:1003C0000034013426082A02031C0034031D0134C2
:1003D00027082B02031C0034031D013428082C02BB
:1003E000031C0034031D013429082D02031C0034B2
:1003F0000134A71F013400342A080319842A26086F
:100400000319FC2A27082B06CF00A717AB17CC012E
:100410002708C9002808C7002908C8002D08C802F5
:100420002C08031C2C0FC7022B08031C2B0FC9021E
:10043000C901C701C801031C242A0310A70CA80C7A
:10044000A90CC90C0130CC002A08A602031C2E2AD4
:100450007E304C07A6070318EE2A332A7E304C075D
:10046000A607031CE32A1830CE00C80DC70DC90D1E
:10047000A90DA80DA70DCC0D2D08A9022C08031C51
:100480002C0FA8022B08031C2B0FA7022B0DCC044A
:100490004C1C4C2A4814572A2D08A9072C0803186D
:1004A0002C0FA8072B0803182B0AA7074810CE0B00
:1004B000352A4B1B481C7B2A0310A90DA80DA70D3C
:1004C000CC0D2D08A9022C08031C2C0FA8022B0808
:1004D000031C2B0FA7022B0D4C040139C80703186E
:1004E000C70A0319C90A031D7B2AC90CC70CC80C0B
:1004F000A60A0319EE2ACF1FC9134908A700470807
:10050000A8004808A9000034CB15FF34A801A901B0
:100510002608C9002908A6002708A9002608A70060
:100520009E30A600CF01A71FA12AC909A909A809C1
:10053000A709C90A0319A90A0319A80A0319A70ACE
:10054000CF17CC012708031DC12A2808A7002908B6
:10055000A8004908A900C901CC152708031DC12A14
:100560002808A7002908A800A901CC114C162708C3
:10057000031DC12A2808A700A801CC1527080319C4
:10058000FC2A4C08A602031D031CE32A0310A71B28
:10059000D02AC90DA90DA80DA70DA60BC72AE32ABD
:1005A0004B1B291CF92AC91FF92AA90A0319A80AF1
:1005B0000319A70A031DF92AA70CA80CA90CA60A5F
:1005C0000319EE2AF92A4B15CB1FFF340130A60080
:1005D000A701A801A901CF0DA70CFF34CB14CB1F95
:1005E000FF34FF30A600A700A800A900CF0DA70C7C
:1005F000FF34CF1FA7130034A701A801A901C90127
:10060000A60100346030CB00A001773083168F0044
:100610000515813083129F00043003179E009F014F
:1006200020308400603003138A010221A03084004E
:1006300050308A0102212030840051308A0101218A
:100640008A0104208030A10080308A010E2004300D
:10065000A50023308A01E5208030A100C0308A0146
:100660000E200430A50034308A01E5200230B300AA
:1006700058308A0109218030A10080308A010E2083
:100680000430A50045308A01E5200230B30058301F
:100690008A0109218030A10080308A010E200430B7
:1006A000A50056308A01E5200230B30058308A0197
:1006B00009218030A10080308A010E200430A5007D
:1006C00067308A01E5200230B30058308A010921E1
:1006D0008030A10080308A010E200430A5007830DF
:1006E0008A01E5200230B30058308A0109218A01CD
:1006F00004208030A10080308A010E200430A50043
:1007000089308A01E5208030A100C0308A010E20A6
:100710000430A5009A308A01E5208030A100CF3056
:100720008A010E20FE308A01952040308A019520F2
:1007300000308A0195200E308A01952011308A01FF
:10074000952011308A01952011308A0195200A30B8
:100750008A0195201B308A01952000308A0195205E
:100760008A110A24E030D0020130031C013ED1027C
:10077000AD01AC011830AB008330AA005108A700CE
:100780005008A6008A0186228A01FC212908D5008A
:100790002808D4002708D3002608D200A901A80100
:1007A0005830A7008330A6005508AD005408AC00AF
:1007B0005308AB005208AA008A01C421013C8A11E7
:1007C0000319EE2B8030A100C8308A010E200430BE
:1007D000A500AB308A01E5208A11032C8030A100EE
:1007E000C8308A010E205508C2005408C1005308C1
:1007F000C0005208BF0002308A0115200430A50055
:10080000B7308A01E5200230B30026308A01092181
:100810008A01B02B89309F000130B300FE308A017D
:1008200009219F148A119F1C172C8A01122CD101B7
:10083000D0011E08D10083161E088312D0000800C4
:1008400063008A01202C45006C0065006B00740079
:1008500072006F006E006900630061005300740055
:1008600079006E0075000000200045005300520022
:100870002D004D00650074006500720020005600D8
:1008800031002E003200200000006C0065006B007B
:10089000740072006F006E00690063006100530015
:1008A000740079006E0075007300000065006B0035
:1008B000740072006F006E006900630061005300F5
:1008C000740079006E00750073002E0000006B004C
:1008D000740072006F006E006900630061005300D5
:1008E000740079006E00750073002E006200000035
:1008F000740072006F006E006900630061005300B5
:10090000740079006E00750073002E0062006500AF
:10091000000020004500530052002D004D006500EE
:100920007400650072002000560031002E00320075
:10093000200000002000200045005300520020004D
:100940003D002000200020002C002000200020007E
:100950002000200000004F00700065006E002000A5
:1009600020002000200020002000200000002000A7
:100970002000200020002000200020002000200077
:02098000000075
:02400E00D43F9D
:00000001FF
